:1074000080E189BD82E189BD09B400FEFDCF089508
:10741000D0D569F08091E9008F931092E900A5D44E
:1074200083FF01C024D58F9187708093E900089570
:107430008EEF0090E10008220092E1000895F20131
:10744000F999FECFF2BDE1BD0895F9DFF89A80B554
:1074500008C0F5DF1FBA80BD0FB6F894FA9AF99A02
:107460000FBE31962F010895E0E0F0E085919491F0
:107470000196089580EE8BB98BEA34D01092890082
:107480008AEF8093880082E080936F0083E080938E
:107490008100E7E5F7E785913AD0E336E1F781E04F
:1074A0008093D7008AE482BF1092D8001092E20045
:1074B0001092DA001092E10080E808D019BC1EBAE0
:1074C0001092E00068D489E059D481E98093D80013
:1074D0000895A3E6B1E090E81AD08D939A95E1F76C
:1074E000089586E008D010C083E005D08F2F0FD01C
:1074F0008E2F0DD080E05E9A729809C005D085E08D
:10750000FADF05D080FDFDCF729A5E9808958EBD9A
:107510008DB587FFFDCF8EB508958FE08221E9F705
:10752000F3DFE3E6F6E090EB5C98892FF0DF80E193
:10753000EEDF5C9A8191EBDF83E68E278F77D1F7C0
:107540009395983B89F70895E3E6F1E097FC38C0FE
:1075500094FC4FC092FE08958684882011F49924EB
:1075600059C0F894C089D78520E030E080E090E4ED
:10757000AFEFBFEF119688199040E0F72D01BD4F96
:107580008D0127FD13C0E0E0F8E011928EE78193B2
:1075900092E4E11791939AE508F092E4E334C9F795
:1075A00081931082BDDFFE0121969EDF92DFF901FB
:1075B00003D520583F4F040D151D8A9411F716C2AC
:1075C0008301282D60906C0170906B0141D019F4FB
:1075D0008823C1F70895380188243AD0B9F58091FD
:1075E0006A01821709F4830160906E0170906D0149
:1075F000F4CF60906E0170906D012AD059F4882309
:10760000C1F708959FEF95FC03C096FE089591E0A1
:1076100097FB890E662477248301222719D0B1F4C1
:107620008823A1F380916A0136F0881650F48217FE
:1076300030F0213003C0881520F4281710F483019E
:10764000282F60906E0170906D01E8CF3801822E76
:10765000F3014ADF3EDFC3E6D1E0E0E5F7E709905A
:107660008591081621F4E735D1F7088080104CCFBA
:10767000C9E031DFCA95E9F7D0E195FC1EC097FC5F
:1076800053C094FC35C0C3E6D2E0E3E6F6E098E0F0
:1076900088E78E0F00840192E817E1F7884F099080
:1076A0000192E817E1F7C858DF4F9A9589F735DF5F
:1076B000C85FD340C33E49F749C0C3E6D6E0EBE517
:1076C000FAE098E08E2F885702900086E817E1F7DD
:1076D00038960A900292E817E1F73897C857D040D9
:1076E0009A9581F71ADFC850DC4FC33E41F72EC090
:1076F000A3EEB6E0E3E6F6E09AE0C6E00D90808106
:107700008025807F802582958193A336B90709F46F
:10771000B2E0E336F90709F4F2E0E336FC0771F76B
:10772000FCDEDA9529F712C0A3EEB9E0E3E6FAE051
:1077300092E00E90829180258F70802582958083C3
:10774000E336F907B1F7E9DEDA9571F7882708958E
:1077500041524455424F59D5F08D14A1C881CFD91B
:10776000F1AF000000FFFFCFCFFFFFFFFFCFCFFF44
:10777000FF0000FE067E7E06FE46565616FE0656A4
:10778000461EFE3F61E9E3FFE3EBE3FFE3EBE3FFCC
:04779000E16B3F006A
:10779400120110010200000841233600010000001C
:1077A400000109023E0002010080320904000001C8
:1077B4000202010005240010010424020405240629
:1077C4000001070582030800FF09040100020A0002
:1077D40000000705040210000107058302100001E0
:1078000011241FBE04B714BE88E18093600010925B
:1078100060008EEF9AE09EBF8DBF222433242101A9
:107820004394310141018AC00F928F939F931F921D
:107830000FB60F9211244F936F938091DA0080FF5F
:1078400037C023C00F920FB68F939F93EF93FF9390
:1078500088278093850080938400E0E5F1E09281A1
:10786000907261F490818917980B908309F45D9A66
:1078700091818917980B918309F4289A239411F424
:107880008315381EFF91EF9154C08091D80080FF7E
:107890000FC08091DA008E7F8093DA008091D9004A
:1078A00080FF04C0ADDD81E08EBB02C019BC1EBAF2
:1078B0008091E10080FF0BC05BD280FF08C05BD2EB
:1078C0008091D800806202DE19BC85E08EBB809179
:1078D000E10084FF1AC04CD284FF17C091DD809173
:1078E000D8008F7DF3DD8FEEA4DD42D28F7E8160E4
:1078F00045D280915301882331F48091E30087FDC4
:1079000002C081E001C084E08EBB8091E10083FF72
:107910000CC02ED283FF09C087EF8BDD82E08EBBC7
:107920001092530185DD27D236D26F914F910F907F
:107930001F909F918F910FBE0F90189580E88093B4
:10794000610010926100B1E0B5BF82E085BF81EFB8
:1079500085B987EE84B984E08DB984E48EB910BA14
:1079600080EF81BB80E68BB980EF8AB980E58CBD62
:10797000BDBDA0E0E4E9F7E705900D92A035E1F781
:107980001D92BB30E9F701FD09C000FF07C07C9BD9
:1079900005C05BDD882312F067DD41F56BDD78946F
:1079A00057DE71F0ABE9B7E0E3E6F7E790E1059069
:1079B0000D929A95E1F7A059BF4FE339B9F7B1DDC0
:1079C00052D026DD80915201807861F48FB180958C
:1079D000807F66991C9B8460982E14DE8110B4DD34
:1079E00092FC02C0332062F73FDD51F3F89489EB3B
:1079F00079DD81E08093E00010926F0010928100A9
:107A0000109285001092840081E085BF15BE2E9AE9
:107A10002F9A2D9A5D9A289A0C940000A4D107C041
:107A200057D102C0C6D239F0A0D182FFFBCF85FF6B
:107A3000F7CF8091F1000895082E83E095D185FD60
:107A400007C08AD102C0B5D269F08FD180FFFBCFC9
:107A50000092F10080915201807221F45D9884E6D9
:107A60008093500108957FD182FF34C180915201EB
:107A7000807221F4289884E680935101CFDF182F7B
:107A8000853431F422248EE7382ED9DC8DE00BC109
:107A9000843511F4C3DFFACF8C34C1F38035B1F3F0
:107AA000843721F484E4C8DF80E0FDC0813611F41E
:107AB00089E5F9C0813429F4B1DF582EAFDF482EB3
:107AC000E5CF803711F483E5EEC0833539F4E0E586
:107AD000F7E78591B1DFE735E1F7E6C0863521F4B8
:107AE00081E3AADF86E3DFC0863761F481E3669B2A
:107AF0008E5F1C9B8F5FA0DF8FB1809582958F700A
:107B00008F5BD1C08837A9F489DF80935201289A0E
:107B100084FD28985D9A83FD5D982E9A81FD2E98AC
:107B20002F9A82FD2F982D9A80FD2D9887FD88240D
:107B3000ADCF8A3649F48FE9DEDCC3E0E8DC7CDFD8
:107B4000CA95E1F7E1DCB0C0833731F487E874DF30
:107B500085E972DF8EE1A7C0853639F4E0E8F3E706
:107B60003ED2E058F040E0F791CF823631F489E51B
:107B700063DF80E061DF80E896C0823419F08736E9
:107B800009F07DC033244ADFD82F48DFC82F46DFF5
:107B9000082F8354843008F085C0063411F4440C57
:107BA000551CF20110926F001736B9F4033489F4B2
:107BB00083E09BDCACDC8EB51EBC3EDF0DB42197B0
:107BC000D1F7A2DC08C0063411F4859101C03DDC78
:107BD00033DF2197C2F72F014AC00334A9F4E11122
:107BE00004C07FDC88ED81DC89DC7BDC82E07DDC2D
:107BF00015DF0DB48EBDCA95D9F7319689DC7EDCD0
:107C0000DA9569F72F0131C00634F1F49F01F4379A
:107C1000D8F4E5D119C002DF063461F4C0FB46F0A8
:107C2000F43728F4182E81E087BFE89511243296A6
:107C3000082E0AC0043439F4DF01B370AD59B94FCE
:107C40008D93319601C005DC21972AF7043431F475
:107C50002F01F370FE2B49F464DC07C0063429F4CD
:107C60002F01F901F43708F4B8D18DE0E5DE0634D0
:107C700011F45694479482E080936F0015C08237C8
:107C8000E1E049F08634E0E031F08E34E3E019F0D1
:107C9000813531F4E2E0F0E089E087BF849103C0F0
:107CA0008B3111F08FE3C8DE83E0BFDB55D095FF49
:107CB00003C009C07ED171F058D080FFFBCF4CD0FB
:107CC00002C077D139F051D080FFFBCF84E0ADDB2B
:107CD0008BE743C00895E4E5F1E067E090915B0134
:107CE00080915C01913231F0913AE1F58132D1F528
:107CF0005ED181C0823271F48191805B8191844038
:107D000089F580915D0180FD2DC0F89481E080931C
:107D1000E00076CD803231F54AD14BD1E9F08530A3
:107D2000D9F023D083FD18C082FFF7CF04C081DED5
:107D30008193615031F09091F3008091F200892B92
:107D4000B1F7C6DF611549F704C033D129F085309A
:107D500019F00BD080FFF9CF8EE79091E8008923CE
:107D60008093E800089584E060DB8091E800089546
:107D70008091E2000895FCDF8E7F80618093E200B5
:107D8000089582E061EC09D083E061E802D084E0EC
:107D900060E842E103C080E060E042E046DB81E071
:107DA00007D01092ED006093EC004093ED00089531
:107DB0009091EB00892B8093EB00089560E0923066
:107DC00029F0913029F4E0E062E102C0E2E16EE3E3
:107DD000F1E0089580915B0188234CF402C0E9D062
:107DE000C1F3C3DF82FFFBCF73CFE3D091F3BDDFDD
:107DF00080FFFBCFB1CF40916101509162014617E6
:107E0000510520F0462F611509F4A6DF50E022C08D
:107E1000D0D061F1853051F1A8DF83FD59CFA5DFC6
:107E200082FD21C080FF16C03091F3002091F20046
:107E300006C081918093F10041502F5F3F4F411563
:107E400019F028303105A8F350E02830310509F445
:107E500051E082DF4115E1F65523D1F604C0A9D0E7
:107E600029F0853019F081DF82FFF9CF31CFEBE5C2
:107E7000F1E0DFDD8193E336E1F72DDF76DF83FF8D
:107E800091C080915B0190915C01913009F170F09B
:107E90009330F1F0953009F444C0963009F456C09F
:107EA000983009F460C0993059F767C0823841F7BB
:107EB00080915F01B9DA2091EB001092E90077D050
:107EC0002295269521702093F1001092F10052C066
:107ED000882311F08230A1F68F71823089F680916B
:107EE0005D018823D1F420915F01277049F220932E
:107EF000E9008091EB0080FF10C0933011F480E224
:107F00000BC080E155DF81E0880F2A95E9F7809367
:107F1000EA001092EA0088E04BDF1092E90047D0B7
:107F20002AC0882391F410915D0110680FB7F8946E
:107F30003ED050DF1ADF80FFFDCF1093E3001038F2
:107F400083E009F482E08EBB0FBF2CC080588230E2
:107F500048F580915D0190915E0130DF603011F154
:107F600026D049DF1FC08038E9F421D08091530129
:107F70008093F100F1DE2EDF15C0882399F49091F3
:107F80005D01923078F49093530111D023DF8091FA
:107F90005301882321F48091E30091E087FD94E070
:107FA0009EBBEFDEE2DE83FF089580E201DF87EF14
:107FB000D4CE8EB388230895A3E6B1E0F437B8F4A5
:107FC0000ED090E40D901D9081E087BFE895329629
:107FD0009A95C1F71124E058F04085E001C083E094
:107FE00001D081E187BFE89507B600FCFDCF089579
:067FFA003136DFCFFBDC95
:040000030000740085
:00000001FF
